:1000000085C09FC082C29DC09CC09BC09AC099C041
:1000100098C07DC896C095C094C093C092C091C04E
:1000200090C08FC08EC056C75CC712C7E2C6E1C67B
:1000300069C7DFC6DEC6DDC6DCC6DBC6DAC6D9C622
:10004000D8C6D7C670C775C778C77DC783C78BC7E3
:1000500091C732C798C730C796C795C794C732C7EC
:10006000C8C6C7C6C6C6C5C6C4C6C3C6C2C6C1C63C
:10007000C0C6BFC6BEC6BDC6BCC6BBC6BAC6FCC629
:1000800004030904120345006E00740072006F003F
:1000900044006500760016035500530042002D0011
:1000A000410056005200490073007000084156524A
:1000B0004953505F32001201010102000008C016CE
:1000C000E105000101020001090243000201008074
:1000D00019090400000102020100052400100104B6
:1000E00024020205240600010524010301070583FB
:1000F0000308006409040100020A0000000705016A
:1001000002080000070581020800000011241FBE3C
:10011000CFE5D4E0DEBFCDBF10E0A0E6B0E0E2E086
:10012000F3E102C005900D92AE38B107D9F713E0A4
:10013000AEE8B0E001C01D92AE31B107E1F74CD896
:10014000DFC85ECF85B78C6085BF8BB780688BBFFB
:1001500083EC8093EE028093E30208951F93DC0109
:10016000162F8091630084FF1EC08091E30298E8FF
:1001700089278093E302112369F01150E4EEF2E045
:10018000212F30E01F5F2B513D4F8D918193E2175E
:10019000F307D9F784EE92E0612FB3D11C5F10937F
:1001A00063001F9108958AE580936300E4CF1F9355
:1001B000DC01162F8091620084FF1EC08091EE0248
:1001C00098E889278093EE02112369F01150EFEE31
:1001D000F2E0212F30E01F5F20513D4F8D91819340
:1001E000E217F307D9F78FEE92E0612F8AD11C5FF7
:1001F000109362001F9108958AE580936200E4CF16
:10020000FF920F931F93CF93DF936091FE02161618
:100210006CF58091FB02CCE0D0E0C81BD109CE5F29
:10022000DC4F63508091FA028F3F09F48CC08D320D
:1002300079F080918E0087FD11C0CE0134D88F3FB8
:1002400009F4C8C0882309F48EC090E080E008C09B
:100250008AE580936100683009F4A1C090E880E0ED
:1002600090938E00809360001092FE028091610056
:1002700084FF27C0809160008F3F19F1182F8930CB
:1002800008F058C0811B8093600080918E0080FD33
:1002900028C02BE4F22E8F5F80938E0087FD28C04C
:1002A000112309F053C004E089ED92E0612F29D1B8
:1002B000183019F08FEF80936000F092D80200930D
:1002C00061009AE080B38C7031F49150D9F71092AC
:1002D000FF021092F902DF91CF911F910F91FF90D1
:1002E000089593ECF92E8F5F80938E0087FFD8CF0F
:1002F000C091FC02D091FD0286FD38C0112399F017
:100300001150DE01E9EDF2E0412F50E01F5F9A014C
:1003100026523D4F8D918193E217F307D9F74F5F36
:100320005F4FC40FD51FD093FD02C093FC02012F75
:100330000C5FBACF18E0811B8093600080918E0023
:1003400080FDCFCFA6CFCE01A1D78ECF89ED92E091
:10035000612FBCD7182F893008F49CC08FEF809391
:1003600060000EE1AACF90E08FEF7ACF1123D9F28F
:1003700011509E01A9EDB2E0612F70E01F5FAB014B
:1003800046525D4FF90184918D932F5F3F4FA41723
:10039000B507C1F76F5F7F4FC60FD71FC4CF8881E6
:1003A000807669F521EE32E01092E102898188239E
:1003B000B9F41092E2023093FD022093FC0290E81F
:1003C00022E08F81882321F48E81821708F448CFA0
:1003D000822F46CF8EE18093610090E08FEF40CF77
:1003E0008530C9F08630E9F0883051F1893089F1E3
:1003F0008A30E9F18B3099F190E820E0E2CFCE012C
:10040000D6D6282F90E82F3FE1F6888187FD15C0CA
:100410008FEF9F7725CF8A818093FF0290E820E0BD
:10042000D0CF8B818130C9F18230B9F1833031F185
:10043000813299F190EC20E0C4CF8E819F7710CF6C
:1004400081E093E09093FD028093FC0290E821E02C
:10045000B8CF8A818093010390E820E0B2CF83EC8B
:100460008093EE028093E30290E820E0AACF3093DD
:10047000FD022093FC0290E821E0A3CF8A8188232B
:1004800089F480E890E09093FD028093FC0290EC68
:1004900024E097CF082F0C5F07CFCE016DD6282F11
:1004A00090ECB1CF813059F0823021F686E990E0AE
:1004B0009093FD028093FC0290EC26E182CF84E8C9
:1004C00090E09093FD028093FC0290EC22E179CFC2
:1004D000A82FB92F8FEF9FEF41E050EA615070F0E5
:1004E0002D9138E0722F782796958795269570FF85
:1004F00002C0842795273A95A9F7F0CF809590956B
:100500000895E6DF8D939D930895CF93CFB7CF9352
:10051000829BFECF829B09C0829B07C0829B05C045
:10052000829B03C0829B01C09EC0DF93C091FB02EF
:10053000DD27CE5FDC4F829B02C0DF91EBCF2F9394
:100540000F931F9300B32FEF02FB20F94F933F93BC
:1005500010B34FEF012702FB21F93BE031C04E7F82
:10056000012F10B3216028C0102F4D7F22600000A2
:1005700000B329C04B7F2460012F000010B32BC0B3
:1005800010B3477F28602AC04F7E00B320612CC083
:100590004F7D10B320622FC04F7B00B3206432C068
:1005A000422700B349934FEF0000102712FB20F9B8
:1005B00010B31C70A9F1297F91F2012702FB21F9E8
:1005C00000B3237F89F23150F0F1102712FB22F99A
:1005D00010B3277E79F2012702FB23F92F7C81F2E9
:1005E00000B3102712FB24F92F7971F200C010B369
:1005F000012702FB25F92F7359F200C000B3102721
:1006000012FB26F9223040F200C010B3012702FB92
:1006100027F9243028F64F77206810B30000F9CF6F
:100620003B503195333010E81ABFB8F0C31BD040AF
:100630000881033C99F10B3489F11981412F1F770F
:100640002091F902121731F40936E9F10D32C1F0A7
:10065000013EB1F02227209300033F914F911F915B
:100660000F912F91DF91CF91CFBFCF9118953091FE
:10067000630034FD56C000936300C3EED2E055C062
:1006800047FD0FEF009300033F914F911F910F9192
:100690002F91DF91CAB7C7FD3BCFE5CF0091000393
:1006A0000023D9F21091FE021123B9F53430BAF1CA
:1006B0003093FE020093FA021091FB023BE0311BE3
:1006C0003093FB022CC00091FE02013034F50AE5A4
:1006D00047FD09C03091610034FD23C000936100E3
:1006E000C8EDD2E022C01A8110FDC1CF3091620066
:1006F00034FD17C000936200CEEED2E016C005278D
:1007000010E002BB1FC0052722C0052727C0052710
:100710002CC0052710E002BB33C04AE503C042ED00
:1007200001C0432FC4E1D0E032E011B31C60929AC3
:1007300002B311BB5F935CE020E820FF052702BBFA
:10074000279517951C3FD8F620FF0527279502BB54
:1007500017951C3FC0F620FF05272795179502BB6C
:100760001C3F98F620FF0527279517951C3F02BBD5
:1007700070F600C0499120FF052702BB2795179509
:100780001C3F38F620FF0527279502BB17951C3F15
:1007900038F520FF05272795179502BB1C3F10F55C
:1007A00020FF0527279517951C3F02BBE8F4242F4F
:1007B0003A9519F6037F5F9102BB00C01091FF02CA
:1007C000C651D04011F01093F90210E81ABF04602E
:1007D00011B3137F402F437F02BB11BB42BB3DCF00
:1007E0000527D3CF0527D8CF0527DDCFFC015091B2
:1007F0008F00F89425B32F7E319148E037FD1EC05D
:1008000025BB789492B7950F82B7891B87FDFCCFE3
:10081000F894AA9A330F2F7E9B993160789492B7FF
:10082000950F82B7891B87FDFCCFF894AA98415099
:1008300029F7615009F77894832F08952061E0CF5C
:1008400064E0D4DF80E008951F93CF93DF93EC0141
:1008500001966881CBDF182F2881243040F4822F45
:1008600090E0019664E0621B8C0F9D1FBFDF812F1B
:10087000DF91CF911F910895AF92BF92CF92DF92F7
:10088000EF92FF921F93CF93DF93EC015B0188817E
:100890001A81811708F4182FCE010396612FA6DF65
:1008A00065010894C11CD11CE12EFF24888190E0D1
:1008B0008E199F09181619060CF042C010E020E0AE
:1008C00030E02E0D3F1D2D5F3F4FCE01820F931F55
:1008D00061E08CDF982F8981181718F4F601919345
:1008E0006F01A8951F5F212F30E0888190E08E195D
:1008F0009F09281739072CF38981181770F4109273
:10090000900080E990E061E071DFF60181936F0172
:10091000A8951F5F8981181790F3F5011082F601E1
:100920001082298130E02E5F3F4FC901DF91CF91C6
:100930001F91FF90EF90DF90CF90BF90AF90089500
:1009400010E0DACFAF92BF92CF92DF92EF92FF9298
:100950000F931F93CF93DF93EC015B01C42E109292
:100960009300442321F480911B0387FD4AC09881A2
:10097000898175010894E11CF11CF5011082DA806F
:100980008C010115110561F1C0E0D0E011C0C0FD7E
:100990001CC087EFD822D092900080E990E064E0FC
:1009A00025DFF70181937F012196C017D10788F4D5
:1009B000A8958091190380939100809118038093EA
:1009C0009200CC2021F3BED1E6CFF8E0DF2ABAD1E5
:1009D000E2CF0F5F1F4F7501E00EF11E0150104076
:1009E000F701108298012E5F3F4FC901DF91CF912F
:1009F0001F910F91FF90EF90DF90CF90BF90AF903D
:100A000008958DE4809390001092910080911A03D4
:100A10008093920080E990E064E0E8DEA8CFA2989D
:100A2000A498A398AA98AC98AB98AD9864D385B5D0
:100A30008F7E85BDAD9AC598C49A08950F931F9374
:100A40008C01FC018081EBDFF801818154D31F917F
:100A50000F910895CF92DF92EF92FF920F931F9321
:100A6000CF93DF93EC0190917C002981C59AC498C3
:100A7000992341F4B19954C0B1996EC083E0809339
:100A80008F0009C0913019F0923009F06FC0B19B0E
:100A9000F3CF90938F0085B38B7E85BB84B3846145
:100AA00084BBAD9885B5806185BD822F24D320910C
:100AB0008F0092B7920F82B7891B87FDFCCFAD9A4A
:100AC00092B7920F82B7891B87FDFCCFAD988A81C0
:100AD00012D397E0E92EF12CEC0EFD1ED0908F0082
:100AE0000FE184E0C82EA895C7016E817FDE182F24
:100AF0002E812430C0F08D81181701F1AA9A92B787
:100B00009D0D82B7891B87FDFCCFAA9892B79D0DDA
:100B100082B7891B87FDFCCF0023D1F00150E3CFC2
:100B200010928F00B8CF822F90E007966C2D621B39
:100B30008C0F9D1F5BDE8D81181701F780E0DF9120
:100B4000CF911F910F91FF90EF90DF90CF9008957C
:100B500080E065DF80ECF3CF892F82958F709695CA
:100B60009695890F8F5F80938F0095CF933009F40E
:100B700085CF82CF1F93F8D210EF10939000109280
:100B8000910080E990E064E031DE80FF07C0809151
:100B90001C03882391F781E81F91089580E01F913D
:100BA0000895FF920F931F938C01FC01F080029631
:100BB00064E01CDEF8018181882359F0F9E0FF151B
:100BC00010F02AE0F22E8F2DD5DF1F910F91FF90AC
:100BD00008958F2D90D280E01F910F91FF9008957E
:100BE0006F927F928F929F92AF92BF92CF92DF923D
:100BF000EF92FF920F931F93CF93DF93EC01062F99
:100C0000F88019818A8180FD7DC064E0762E58E0ED
:100C1000652E002321F480911B0387FD83C0A12E44
:100C2000BF2C6E01EE24FF24450108948108910831
:100C30000BC0E814F90410F097FD6BC00894E11C98
:100C4000F11C0894C11CD11CEA14FB0408F05FC01D
:100C5000A895809119038093910080911803809347
:100C60009200F6018185809393001C810023D1F5C9
:100C7000177FE0FC44C01093900080E990E064E0AE
:100C8000B5DD9A8190FDD5CF892F872169F1F601D5
:100C900011858F81811781F18885811769F18E8196
:100CA000877FE0FC8860809390008B815DD280E933
:100CB00090E064E09BDD811709F4C0CF80911C03B4
:100CC0008823A9F780E8DF91CF911F910F91FF90C2
:100CD000EF90DF90CF90BF90AF909F908F907F90DC
:100CE0006F9008952FD0C7CF962131F08B8142DFCE
:100CF000882309F4A3CFE7CF8B81FDD19FCF186064
:100D000021D0B9CF40E2742E30E4632E82CF80E050
:100D1000DACF8D818093900080E990E064E066DD19
:100D20009A81B2CF8DE480939000109291008091CF
:100D30001A03809392001092930080E990E064E09F
:100D400055DD6DCF8091180390911903A0911A037E
:100D5000B0911B030196A11DB11D809318039093C0
:100D60001903A0931A03B0931B0308952091CC029A
:100D70003091CD028091CA029091CB02281B390B91
:100D8000C90108952091CC023091CD022115310581
:100D9000E1F08091CA029091CB02FC01EF54FE4F2A
:100DA000E08101969093CB028093CA028217930749
:100DB00018F4F0E0CF0108951092CD021092CC0209
:100DC0001092CB021092CA02F4CFEFEFFFEFCF01E7
:100DD0000895CF93DF93C2E0D0E080919900809393
:100DE000B6011092B70190E0FC013197ED32F105A8
:100DF00060F180EC8093B70122E030E08BE18093DA
:100E0000B101809195008093B2011092B3012093BB
:100E1000B4018EE08093B5011092CB021092CA0209
:100E200088E090E09093CD028093CC02E1EBF1E07A
:100E300090E081919827215030408FEF2B3F380769
:100E4000C1F79083DF91CF910895ED5EFF4F099434
:100E5000E0919A00EA3909F49FC0E63909F4A9C083
:100E6000E73909F4A9C0F0E0EF71F070EC59FF4FD9
:100E7000E081E093B801C3E09E018BE18093B10172
:100E8000809195008093B2013093B301C093B40177
:100E90008EE08093B5011092CB021092CA02CE016F
:100EA00006969093CD028093CC02019709F0BECFB5
:100EB000E1EBF1E090E0C5CF8AE990E0C1DC8093FE
:100EC000B7019ACF8AE990E067EB71E0D5DCEC01DD
:100ED0002196D2CF88EB91E06CEA70E00AD2CBE0A9
:100EE000CBCFE0919A0020919B00E63909F458C0DD
:100EF000E73909F45CC0F0E0EF71F070EC59FF4F96
:100F000020837ACF80919A0080931B0380919B006D
:100F100080931A0380919C008093190380919D0017
:100F20008093180369CF8AE990E094DD8093B7013C
:100F300063CF8AE990E082DD5FCF8AE990E031DE1D
:100F40008093B70159CF8AE990E060E049DE809351
:100F5000B70152CF8AE990E067EB71E040E0F2DC44
:100F6000EC01219689CF8AE990E061E039DE809337
:100F7000B70142CF8AE990E067EB71E041E0E2DC43
:100F8000EC01219679CF8AE990E05EDC8093B8018C
:100F90001092B901C4E070CF89EC8093B7012CCFD7
:100FA00085B5922F9770887F982B95BDA4CF23BDD0
:100FB000A2CFE5B5E7705DCFE3B55BCF282F809179
:100FC0001D03882359F41092AE011092AD012B310C
:100FD00009F46DC088EC80931D0308958091AD01E4
:100FE0009091AE01009799F331E08931930708F0B1
:100FF00056C0FC01EC56FF4F2083FC013196F09364
:10100000AE01E093AD01E430F10509F45CC0E530D8
:10101000F10509F441C0E530F105E0F28091AF013E
:101020009091B001E817F907A9F6A4E9B0E090E0C3
:101030008D9198273197E1F71092AE011092AD0192
:10104000992309F456C080EB8093B6018093B701D1
:101050008BE18093B101809195008093B201109251
:10106000B30182E08093B4018EE08093B5011092C9
:10107000CB021092CA0288E090E09093CD02809358
:10108000CC02E1EBF1E090E08191982731E0E83B80
:10109000F307D1F790839ECF2E3009F49BCF1092A7
:1010A000AE011092AD0188EC80931D03089520934A
:1010B000940081E090E09093AE018093AD0188ECC4
:1010C00080931D030895809197008093AF018091D4
:1010D00096008093B0018091AF019091B001069687
:1010E0009093B0018093AF018A51914008F472CF80
:1010F000D6CF6FDE6FCF982F969596958F5F891B11
:1011000080931C0380911C038823E1F70895789451
:101110001F920F920FB60F9211248F93F894809123
:101120001C03882329F080911C03815080931C03A9
:101130007894F8948091840081508093840088236F
:1011400061F489E48093840080911D03882329F051
:1011500080911D03815080931D0378948F910F908F
:101160000FBE0F901F901895982F9F5F86958695BC
:10117000981B90931C030895FC018091D70288234B
:1011800041F48381813051F028EC30E083E490E039
:1011900009C020E030E080E090E004C026EB30E0C1
:1011A00082E190E03093FD022093FC020895FC015F
:1011B00080818076803219F080E090E008958091FF
:1011C000D7028823C9F7818180528230A8F7109214
:1011D000D6028FEF90E00895EF92FF920F931F9346
:1011E000CF93DF9388E190E02EE00FB6F894A895B6
:1011F00081BD0FBE21BD82E188BB84E387BB80E255
:1012000085BB84BB12BA8CE081BB11BA83E083BF7B
:1012100081E089BF85E090E09BBD8ABD80E18FBD04
:1012200089E08EBD85BD82E083BD8CD77894009126
:10123000D7028EECE82E82E0F82EA895E1D70023A5
:10124000E1F78091620084FFF8CFC0E0D0E01C2F6E
:1012500099DD97FD0FC0FE01E253FD4F8083612FA2
:101260006F5F2196C830D10591F760938500C70163
:101270009ED7E3CF6C2FCC23C1F7809185008823C4
:10128000E1F260938500C70192D7D7CF1F93CF9328
:10129000DF93EC01162F899191DE1150E1F7DF9178
:1012A000CF911F9108959C018091D602882359F413
:1012B0008BE48093EE02A6E8B0E0F90187E00190AC
:1012C0000D928150E1F781E090E008959C018091BA
:1012D000D602882359F4F901A6E8B0E087E00D9022
:1012E00001928150E1F787E090E0089580E090E07E
:1012F0000895FB01DC0105900D920020E1F70895AF
:02130000FFCF1D
:10130200FF5A5A5A000000000000000000000000CE
:101312000000000001020A0032000180000000000B
:0E13220000000000010180250000000008000E
:00000001FF
